:020000006F2966
:0800080005288D00030E831290
:100010008C000408C7000F18F1288F18FB280F194F
:100020003B298F1948290F1A53298F1A5F290F1B53
:100030001C29910A0319900A1008013C031D262867
:100040001108383C031D2628900191018F011008EA
:10005000031D8B286430110203188B280A3011020B
:10006000031854281108023C031C38280F15A9282E
:100070001108033C031C3E288F15A9281108053CD4
:10008000031C44280F16A9281108063C031C4A2803
:100090008F16A9281108083C031C50280F15A92801
:1000A0000F14861C8E17A9280F1411080A3C031977
:1000B0006928013E03196E28013E03197328013E89
:1000C00003197828013E03197D28013E031982286F
:1000D000A9281430840033088A23A9281930840001
:1000E00034088A23A9281E30840035088A23A928C9
:1000F0002330840036088A23A92828308400370852
:100100008A23A9282D30840038088A230830B200B9
:1001100047088400A9281008031D9228A430110262
:10012000031CA2280F141008013C031DA928110864
:10013000183C0319B228013E0319CC280A3E0319C2
:10014000E928A928B20BA8280F170830B200A9285F
:100150008F146400470884000C0E83008D0E0D0E72
:100160000B110900BC033918D428B918C028391953
:10017000BA28A9288316061083120610B917A928D1
:100180008316061083120610BB0C00000000031C2F
:10019000CA2806143917A928391FA928BA03031930
:1001A000B91006143913A9288316061083120610F5
:1001B0000130432383160614831206304323061CA2
:1001C000E3280314E4280310BB0CBA030319391005
:1001D000A928B91FA928831606148312B913391147
:1001E000A9280000000000000130432386130330DB
:1001F0004323861719280000013043238613033058
:1002000043238617083043230630920014308400BD
:10021000000C850D840A000C850D840A000C850DE8
:10022000840A000C850D840A000C850D840A0000E8
:100230000510920B082919288613033043238617CB
:10024000083043230630920014308400800C850D62
:10025000840A800C850D840A800C850D840A800C2C
:10026000850D840A800C850D840A00000510920B10
:1002700026290510192849234923861301304323D1
:1002800086171E304323861301304323861719280F
:1002900049230000000086132030432386170130D5
:1002A00043238613192849238617013043238613D5
:1002B0001E3043238617013043238613192800007C
:1002C000000086170130432386130130432386172D
:1002D0001C304323861301304323861719288316C5
:1002E00000308500831200308500831607308600B9
:1002F00083128030860083165F308100831289016B
:100300004A2381010B118B168B1739153919862950
:10031000CC30BB000830BA00B914B9188D2944306C
:10032000BB000830BA00B914B91894293230BC00A7
:10033000BC08031D9829391539199C29CC30BB00FC
:100340000830BA00B914B918A329BE30BB00083070
:10035000BA00B914B918AA290830BA0039143918E2
:10036000AF29861CB529CF0BD2290430CF003B081A
:10037000BE000330C400BE1FC129C4173E08003CA4
:10038000BE000310BE0CBD01EC224108C300C20137
:10039000C1010A30B3003430C8000F230C30B7005D
:1003A0000D30B800143096223C3096220C30962244
:1003B000A622BD1BD6295C309622A622BF00A6220B
:1003C000C000A6223F08BE004008BD004C30C0005F
:1003D000D930BF00C6224008C9003F08CA00BE018C
:1003E0003B08803EBD000030C000D930BF00C622AF
:1003F0003F08C0004208BF004908BE004A08BD00CF
:10040000B8220030C0008E30BF00B9223E08C900BB
:10041000C0003D08CA00BF002C30BE007E30BD00C9
:10042000B8223E08CB003D08CC000230C000E930C5
:10043000BF00C6223F08BE004208BD00B630C00063
:100440000530BF00B9224B08C0004C08BF00C622CF
:100450004008BE003F08BD000330C000C630BF00EA
:10046000B8223E08CB003D08CC0086185A2A49081D
:10047000BD004A08BE00EC224108C300C600400887
:10048000C2003F08C1000430BD00C10CC20CC30C47
:10049000BD0B452AC1010430C4003330C8000F230E
:1004A0000F30B70046080F39B8005030BC00BC0808
:1004B000031D572A8E1F622A4B08CD004C08CE0020
:1004C00072238E134B08BE004C08BD004D08C000BF
:1004D0004E08BF00B8220530C400BE1F792A3D086F
:1004E000BF003E08C000C0224008BE003F08BD005B
:1004F000C4173D08BF003E08BD003F08BE00EC2207
:100500004108C3004008C200C1013330C8000F23B6
:100510000E30B800852986112030BD0006168616DB
:1005200000008612BD0B8F2A86150800BD008611BB
:100530000830BE008616BD1F9F2A0616A02A061286
:10054000BD0D8612BE0B9A2A86150800861108304A
:10055000BE00861600000000061DB02A0314B12A52
:100560000310BD0D8612BE0BA92A86153D08080092
:10057000C0223F08BD070318BE0A4008BE0700346A
:10058000BF09BF0A0319C003C0090034D222C40C3A
:10059000C30C0318DB22C00CBF0CC20CC10CC50B72
:1005A000C72A00341030C5004008C4003F08C3000B
:1005B000C001BF0100343D08BF070318C00A3E0850
:1005C000C00700348B2224309622EF30962234303C
:1005D0009622AF309622080003101030C200BF01EF
:1005E000C001C101BE0DBD0DC10DC00DBF0DC20BBF
:1005F000FA2A00344130840004234030840004236C
:100600003F3084000423F22A03300007C300C319DB
:10061000800030300007C300C31B8000003448084E
:1006200084000F304405063CC5003B23C50B152B49
:100630000F304405C500C41F282B4508023C031990
:10064000252B0F3041050319282BC4130B30352BF4
:10065000410E0F39031D342B441B342B45030A3044
:10066000031D352B0030352B44178000840A3B23B3
:10067000C50B1B2B08000430C000C30DC20DC10DFB
:10068000C00B3D2B080092000000920B442B080089
:10069000080008008E0101308F00900191010830A0
:1006A000B2000617E222662303308A00B901013046
:1006B000CF001030B3001130B4000130B500093064
:1006C000B6000930B7000930B800080089016D2371
:1006D000CD00890A6D23CE0008008316081483120A
:1006E000080808004D0889017A23890A4E087A23F0
:1006F00083120800880083168B1388010815553073
:100700008900AA30890088148B178818852B081156
:100710008312080092009207920792079207053011
:1007200093001208A5238000840A920A930B912B50
:020730000800BF
:06074A0082073E34513429
:10075000493445343E34003442347F34403400342C
:1007600042346134513449344634213441344534BF
:100770004B3431341834143412347F341034273469
:1007800045344534453439343C344A3449344934A9
:100790003034013471340934053403343634493487
:1007A00049344934363406344934493429341E3402
:1007B0000034003400340034003408340834083481
:1007C00008340834003407340534073400343E3428
:1007D00041344134413422347C34043418340434F8
:1007E0007834003460346034003400343E344134B2
:1007F000413441343E347F340834083408347F3483
:00000001FF
